:0200000480007A
:100000006F000005732F2034930F80006308FF03F7
:10001000930F90006304FF03930FB0006300FF038E
:10002000130F000063040F0067000F00732F2034CC
:1000300063540F006F00400093E19153171F0000BD
:1000400023223FFC171F000023200FFC6FF01FFF2F
:100050009300000013010000930100001302000050
:100060009302000013030000930300001304000038
:100070009304000013050000930500001306000020
:100080009306000013070000930700001308000008
:10009000930800001309000093090000130A0000F0
:1000A000930A0000130B0000930B0000130C0000D8
:1000B000930C0000130D0000930D0000130E0000C0
:1000C000930E0000130F0000930F0000732540F102
:1000D0006310050097020000938202017390523072
:1000E000735044749702000093820201739052305F
:1000F00073500018970200009382020273905230EE
:10010000B70200809382F2FF7390023B9302F001EA
:100110007390023A7350403097020000938242017C
:100120007390523073502030735030309301000080
:1001300097020000938242ED739052301305100035
:100140001315F501634C05000F00F00F930110002B
:100150009308D0051305000073000000930200000F
:10016000638A020073905210B7B20000938292101B
:100170007390223073500030970200009382420146
:1001800073901234732540F17300203093012000E6
:100190009300000013A7000093030000631277266A
:1001A000930130009300100013A710009303000088
:1001B00063187724930140009300300013A7700068
:1001C00093031000631E7722930150009300700088
:1001D00013A730009303000063147722930160009B
:1001E0009300000013A7008093030000631A772098
:1001F00093017000B700008013A700009303100064
:100200006310772093018000B700008013A700805F
:10021000930310006316771E930190009300000073
:1002200013A7F07F93031000631C771C9301A000B9
:10023000B70000809380F0FF13A700009303000035
:100240006310771C9301B000B70000809380F0FF2B
:1002500013A7F07F930300006314771A9301C00083
:10026000B700008013A7F07F93031000631A77187C
:100270009301D000B70000809380F0FF13A70080A7
:1002800093030000631E77169301E00093000000C3
:1002900013A7F0FF93030000631477169301F00097
:1002A0009300F0FF13A7100093031000631A771454
:1002B000930100019300F0FF13A7F0FF93030000E8
:1002C00063107714930110019300B00093A0D00045
:1002D0009303100063967012930120011302000033
:1002E0009300F00013A7A0001303070013021200ED
:1002F00093022000E31652FE930300006312731072
:1003000093013001130200009300A00013A7000125
:1003100013000000130307001302120093022000D1
:10032000E31452FE93031000631C730C930140010D
:10033000130200009300000113A7900013000000B7
:1003400013000000130307001302120093022000A1
:10035000E31252FE930300006314730A93015001E9
:10036000130200009300B00013A7F0001302120064
:1003700093022000E31852FE9303100063127708E3
:1003800093016001130200009300100113000000AC
:1003900013A780001302120093022000E31652FEFE
:1003A00093030000631E77049301700113020000A1
:1003B0009300C000130000001300000013A7E0002A
:1003C0001302120093022000E31452FE9303100064
:1003D00063187702930180019320F0FF93030000DC
:1003E0006390700293019001B700FF009380F00FBB
:1003F00013A0F0FF93030000631470006310300239
:100400000F00F00F638001009391110093E1110040
:100410009308D00513850100730000000F00F00F52
:10042000930110009308D00513050000730000002D
:0C043000731000C000000000000000007D
:1010000000000000000000000000000000000000E0
:1010100000000000000000000000000000000000D0
:1010200000000000000000000000000000000000C0
:1010300000000000000000000000000000000000B0
:081040000000000000000000A8
:040000058000000077
:00000001FF
